:020000040800F2
:1040000000100020317200089D7100089F710008A7
:10401000A1710008A3710008A5710008000000004C
:10402000000000000000000000000000A771000870
:10403000A971000800000000AB710008AD71000814
:1040400079720008797200087972000879720008A4
:104050007972000879720008797200087972000894
:104060007972000879720008797200087972000884
:104070007972000879720008797200087972000874
:104080007972000879720008797200080000000057
:10409000000000000000000000000000797200082D
:1040A0007972000879720008797200087972000844
:1040B000797200087972000879720008B1710008FD
:1040C000797200080000000000000000797200080A
:1040D00079720008BD710008C97100087972000882
:1040E00079720008797200087972000800000000F7
:1040F00000000000000000000000000000000000C0
:1041000000000000000000000000000000000000AF
:10411000000000000000000079720008D57100085E
:10412000000000000000000000000000000000008F
:10413000000000000000000000000000000000007F
:10414000000000000000000000000000000000006F
:10415000000000000000000000000000000000005F
:10416000000000000000000000000000000000004F
:10417000000000000000000000000000000000003F
:10418000000000000000000000000000000000002F
:10419000000000000000000000000000000000001F
:1041A000000000000000000000000000000000000F
:1041B00000000000000000000000000000000000FF
:1041C0000000000000000000000000005FF808F19F
:1041D00010B5054C237833B9044B13B10448AFF341
:1041E00000800123237010BD70000020000000003B
:1041F0008C83000808B5034B1BB103490348AFF398
:10420000008008BD00000000740000208C830008BE
:1042100038B50E4B054618784FF47A73B3FBF0F3BC
:104220000B4A1068B0FBF3F000F0BEF9044658B931
:104230000F2D09D8024629464FF0FF3000F074F9DF
:10424000044B20461D6038BD012038BD0000002011
:10425000080000200400002008B5032000F052F9F7
:104260000020FFF7D5FF02F099FE002008BD0000F6
:10427000034A044B11681B780B441360704700BF5E
:104280004401002000000020014B1868704700BF67
:104290004401002038B50446FFF7F6FF0546631CCD
:1042A0001EBF044B1B78E418FFF7EEFF401B84424F
:1042B000FAD838BD00000020002373B5019390F8B0
:1042C0002430012B74D001234D6880F82430062D52
:1042D00002684FEA85030C6825D82B441F25566BCE
:1042E000053B9D4026EA050504FA03F32B4353637F
:1042F000092C4FEA44038D682FD907262344D1683F
:104300001E3B9E4021EA060105FA03F30B43D360EE
:10431000A4F11003012B2BD90023002280F82420C4
:10432000184602B070BD0C2D0BD82B441F25166B00
:10433000233B9D4026EA050504FA03F32B43136350
:10434000D6E72B441F25D66A413B9D4026EA05054A
:1043500004FA03F32B43D362CAE707261169234407
:104360009E4021EA060105FA03F30B431361CFE7F0
:10437000104B9A4216D193681B02CDD49368102C2F
:1043800043F400039360C7D10B4B0C4A1B68B3FB8B
:10439000F2F20A2353430193019B002BBCD0019BF3
:1043A000013BF8E7836A43F0200383620123B4E70B
:1043B0000223B5E7002401400800002040420F001E
:1043C00038B5036804469A68D20701D4002038BD86
:1043D0009A6822F001029A60FFF756FF05462368AB
:1043E0009B68DB07F2D5FFF74FFF401B0228F6D989
:1043F000A36A012043F01003A362E36A43F00103C0
:10440000E36238BD70B50446002871D0836A23B9D1
:10441000C36280F8243002F0E3FD2046FFF7D0FFAE
:10442000A36A13F0100FA36A64D1002862D1E16976
:1044300023F48853626823F0020343F002030A4323
:10444000A168A362E368B1F5807F42EA430238D0F5
:10445000012914BF06464FF480766569012D07D106
:10446000002B30D1A369013B46EA433545F4006691
:104470002368B1F5807F5D6825F4694545EA060546
:104480005D609E681D4D05EA060545EA02059D60D2
:1044900001D0012920D1216901390905DD6A25F4FE
:1044A00070052943D9629968154B0B409A4215D182
:1044B0000023E362A36A23F0030343F00103A36232
:1044C00070BD0E46C9E7A36A43F02003A362E36A06
:1044D00043F00103E362CBE70021DFE7A36A23F0A7
:1044E000120343F01003A362E36A43F00103E362A3
:1044F000012070BD43F01003A362F9E7FDF7E1FF6F
:10450000FE0E1FFF074A0002D36800F4E06023F4A8
:10451000E0631B041B0C43F0BF6343F4003303430D
:10452000D360704700ED00E0174B30B5DC68C4F392
:104530000224C4F10703251D042B28BF0423062DE4
:104540004FF0010598BF002405FA03F303F1FF3390
:1045500088BF033C1940A14005FA04F4013C224005
:10456000002842EA01024FEA0212AFBF00F16040A8
:10457000064B00F00F00D2B2A5BFD2B200F56140E9
:104580001A5480F8002330BD00ED00E014ED00E087
:104590000123420900F01F0003FA00F0014B43F829
:1045A0002200704700E100E00138B0F1807F0AD2BC
:1045B000F021064B064A586082F82310002007229B
:1045C00098601A6070470120704700BF10E000E05B
:1045D00000ED00E090F8213010B5022B03D0042349
:1045E0008363012010BD03681A6822F00E021A606E
:1045F0001A6822F001021A60184A93421FD014323E
:1046000093421ED0143293421DD0143293421DD0D7
:10461000143293421DD0143293420CBF4FF48013D6
:104620004FF080730E4A00245360012380F821303C
:10463000436B80F820407BB19847204610BD012392
:10464000F0E71023EEE74FF48073EBE74FF480536D
:10465000E8E74FF48033E5E7184610BD0800024054
:10466000000002402DE9F74F00221646654BDFF8A7
:10467000A4E1DFF8A4C14FF001080C6808FA06F8BD
:1046800008EA0404A0457FD14D68122D00F0AF80E8
:1046900000F28880022D00F0A7807CD8002D00F069
:1046A0008E80012D00F09E804FF00F09FF2C93BFEC
:1046B000824606F18045083DD0F800B092BFB500B3
:1046C000D0F804B0AD0009FA05F82BEA080802FAA0
:1046D00005F588BF00F1040A48EA0505CAF800504C
:1046E000D1F804A01AF0805F4ED0474D464FAD6917
:1046F00026F0030845F00105BD61BD6908F1804859
:1047000005F00105019508F5803806F0030B019DC1
:104710004FEA8B0BD8F8085009FA0BF925EA09097A
:104720003A4DA84268D005F58065A84266D005F5E7
:104730008065A84264D005F58065A8420CBF0325BA
:10474000042505FA0BF545EA0905C8F808501D6867
:104750001AF4803F14BF2543A5431D605D681AF419
:10476000003F14BF2543A5435D609D681AF4801F78
:1047700014BF2543A5439D60DD681AF4001F14BFD4
:104780002C4325EA0404DC600136102E7FF473AF5D
:1047900003B0BDE8F08F032D22D0112D84D1CA685B
:1047A000043281E71A4FBD4209D012D8DFF86C906D
:1047B0004D4504D009F580394D457FF475AF8A68C1
:1047C000C2B1012A0CBFC0F81080C0F814800822C2
:1047D0006AE77545F3D06545F1D0DFF84490EBE723
:1047E000002261E7CA685FE7CA6808325CE7CA6806
:1047F0000C3259E7042257E70025A2E70125A0E77C
:1048000002259EE70004014000100240000801401C
:1048100000002110000031100000321000001110C3
:10482000000022100AB1016170470904FBE7C36868
:104830005940C16070470268536913F480630DD01A
:104840006FF4806353610423202203640023036315
:1048500080F83C3080F83D200120704718467047B2
:104860002DE9F843044617469946C1F307488EB22E
:104870002568B8F1010F0CBF6B69AB6936EA030319
:1048800014BF0120002008B9BDE8F8836B695A0500
:1048900012D52B68202243F400732B606FF48063E1
:1048A0006B610423236400230120236384F83C30DC
:1048B00084F83D20BDE8F8837B1CD9D04FB9002394
:1048C0002022236384F83C3084F83D200320BDE897
:1048D000F883FFF7D9FCA0EB09008742C8D2EEE7C6
:1048E0002DE9F843044690461F46089EC1F3074948
:1048F0008DB22368B9F1010F0CBF5B699B6935EA82
:1049000003030CBF01230023434502D00020BDE870
:10491000F8837B1CEDD05FB900232022236384F849
:104920003C3084F83D20032084F83E30BDE8F88315
:10493000FFF7AAFC801B8742DBD2EDE770B5044687
:104940000D46164623685B691B0601D5002070BD25
:104950002046FFF770FFA8B96A1CF3D065B9236C35
:10496000202243F02003236400230320236384F8E0
:104970003C3084F83D2070BDFFF786FC801B8542EB
:10498000E0D2ECE7012070BD2DE9FF411546026839
:10499000984613680B9E43F4807313600F4600968D
:1049A0000A9B00224FF001110446FFF799FF68B9F6
:1049B000236807F0FE071F610A9A33461A4920460A
:1049C000FFF74EFF30B1236C042B18D0032004B046
:1049D000BDE8F081236803905A690A9903929B69A4
:1049E000324603932046039BFFF7A8FF48B1236C90
:1049F000042BEBD12268136843F400731360012089
:104A0000E5E7B8F1010F236802D1EDB21D61DEE7E1
:104A10002A0A1A610A9932462046FFF78FFF0028BA
:104A2000E5D12368F1E700BF020001002DE9FF4155
:104A30009846036816461A680B9D42F480621A6015
:104A40001A680F4642F480721A604FF00111009507
:104A50000A9B00220446FFF743FF80B92368FFB298
:104A600007F0FE021A612D492B460A9A2046FFF7ED
:104A7000F7FE40B1236C042B01D1012000E003209C
:104A800004B0BDE8F081236803905A690A99039243
:104A90009B692A4603932046039BFFF74FFF40B1D3
:104AA000236C042BEBD12268136843F4007313606A
:104AB000E3E7B8F1010F236824D1F6B21E612A465C
:104AC0000A992046FFF73AFF02460028E8D12168FC
:104AD00020460B6843F480730B6000950A9B4FF0EF
:104AE0000111FFF7FDFE0028C9D1236847F0010737
:104AF0001F610A9A2B4609492046FFF7B1FE00289C
:104B0000B8D1BDE7320A1A610A992A462046FFF752
:104B100015FF0028C4D12368CFE700BF02000100C1
:104B200070B504460D4616462068436913F04003ED
:104B300001D0002070BD4269D2060BD56FF0100283
:104B400042612022236484F83C302363012084F8EE
:104B50003D2070BD5DB9236C032043F02003236426
:104B6000202384F83D30002384F83C3070BDFFF7EB
:104B70008BFB801B8542D7D2EDE770B504460D460E
:104B8000164623685B695B0701D5002070BD20468F
:104B9000FFF751FEA8B96A1CF3D065B9236C202237
:104BA00043F02003236400230320236384F83C3074
:104BB00084F83D2070BDFFF767FB801B8542E0D283
:104BC000ECE7012070BD000038B5044608B90120AB
:104BD00038BD90F83D3003F0FF021BB980F83C204F
:104BE00002F02CFA2423226884F83D30136823F065
:104BF0000103136001F0A0F863682F4A934230D894
:104C00002E4A9042E3D92E4A2168B0FBF2F24A6064
:104C100001320A62284A0138934232D85B00B0FB65
:104C2000F3F0431CC3F30B03042B38BF0423CB6105
:104C3000226AE369002013430B60E268236913438F
:104C40008B60A26963691343CB600B6843F0010377
:104C50000B602023206484F83D30206384F83E00FC
:104C600038BD184A9042B2D9154D4FF49672B0FB38
:104C7000F5F521686A434D604FF47A75B2FBF5F2A1
:104C8000C6E7A26852B903EB4303B0FBF3F0431C41
:104C9000C3F30B036BB143F40043C8E7192253433A
:104CA000B0FBF3F0431CC3F30B0313B143F44043D5
:104CB000BDE70123BBE700BFA08601007F841E0083
:104CC00040420F00FF083D002DE9F34704469A4695
:104CD000884691460C9EFFF7D7FA94F83D3005467A
:104CE000202B03D0022002B0BDE8F08700901923EA
:104CF00001223E492046FFF7F3FD0028F2D194F847
:104D00003C30012BEED0012384F83C30236800278F
:104D10001A684146D20758BF1A6820465CBF42F065
:104D200001021A601A6822F400621A60212384F8D2
:104D30003D30402384F83E300A9B27646362BDF80F
:104D40002C30019563852A4B0096E362638D4A46B9
:104D500023855346FFF718FE00282AD0236C84F8D9
:104D60003C70042B07D10120BDE7FFF7E7FD20B120
:104D7000236C042B34D00320B5E7616A27684B1CF1
:104D800063620B78228D3B61638D501E013B9BB2A9
:104D900063857B6980B25B0720850AD548B18B1C8F
:104DA00063624B78023A3B61638D2285013B9BB283
:104DB0006385238D2A4631462046002BD5D1FFF747
:104DC000DCFE0028D4D12268136843F4007313601A
:104DD000202384F83C0084F83D3084F83E0082E7CC
:104DE0002268136843F400731360BCE702001000EC
:104DF0000000FFFF2DE9F047044686B09A460D46B5
:104E00009146109FFFF740FA94F83D300646202B5C
:104E100004D00225284606B0BDE8F087009019238B
:104E2000012281492046FFF75BFD0028F1D194F86B
:104E30003C30012BEDD0012384F83C3023684FF047
:104E400000081A682946D20758BF1A6820465CBF76
:104E500042F001021A601A6822F400621A602223EA
:104E600084F83D30402384F83E300E9BC4F84080E7
:104E70006362BDF83C30019663856C4B0097E3623A
:104E8000638D4A4623855346FFF7D0FD054630B172
:104E9000236C84F83C80042B3DD10125BAE7228D98
:104EA000236892B902905A6902929A690292029A10
:104EB0001A6842F400721A60202384F83D300023FF
:104EC00084F83E3084F83C30A4E7012A25D11A68E2
:104ED00022F480621A6072B6236803905A690392C2
:104EE0009A690392039A1A6842F400721A6062B6D1
:104EF000DFF83C81238D002BDED0032B77D8012BEC
:104F000027D1324639462046FFF70AFE00283FD017
:104F1000236C202BC1D103257CE7022A1A680ED10D
:104F200042F400621A6072B6236804905A690492CF
:104F30009A690492049A1A6822F48062D6E742F4CD
:104F400080621A6005905A6905929B690593059BDA
:104F5000CEE7022B00963B464FF00002414620462A
:104F600024D1FFF7BDFC0028D5D172B623681A689A
:104F700042F400721A60626A1B69511C616213700C
:104F8000238D013B2385638D013B9BB2638562B614
:104F9000636A5A1C6262226812691A70238D013B8F
:104FA0002385638D013B9BB26385A3E7FFF798FCE4
:104FB00002460028AFD121680B6823F480630B60A0
:104FC00072B6636A2046591C6162216809691970CA
:104FD000238D0096013B2385638D4146013B9BB2A7
:104FE00063853B46FFF77CFC0028BFD093E7324641
:104FF00039462046FFF794FD002889D1636A5A1C80
:105000006262226812691A70238D2268013B23852F
:10501000638D013B9BB2638553695B077FF56AAF84
:10502000636A591C6162B7E7020010000000FFFFCD
:105030000400010070477047704770477047704721
:10504000704770477047704790F83D3010B5293B66
:10505000012B0446036839D800220263282280F815
:105060003D201A6822F400621A605A6812F4006245
:1050700054D05A68606B22F400625A6090F8213074
:10508000012B394B31D04363FFF7A4FA50B12268AA
:10509000606B136823F001031360202384F83D3014
:1050A000436B984794F83D30282B0ED1236C5B0757
:1050B0000BD52E4B2022E36200232046236384F885
:1050C0003D2084F83E30FFF7BAFF10BD90F83D2038
:1050D000602A05D05A6812055CBF202280F83D2066
:1050E0000022226384F83E20BBE7A06B4363FFF7F6
:1050F00071FA0028D6D022685369580604D5636A2D
:105100001269591C61621A702268A06B136823F03F
:1051100001031360202384F83D30C1E794F83D106B
:10512000602914D1202184F83D1022645A69510667
:1051300004D5626A1B69511C6162137022682046A3
:10514000136823F001031360FFF77DFFAAE75A6994
:10515000520604D5626A1B69511C616213702046B5
:10516000FFF770FF9EE700BF455800080000FFFFF3
:105170000368F0B59D6959695A6890F83E408DB052
:10518000E4B2102C02D0402C40F0568211F0011FE6
:1051900066D0970564D590F83E40402C43D1046D0D
:1051A000002C3BD1446C04F0FE041C61944E954CE1
:1051B0002E400C40002E00F0A281934D0D40002D9A
:1051C00000F06981550540F16681002C40F0638153
:1051D00090F83D20058D90F83E10D2B2C9B2C46A55
:1051E000002D40F01781212A40F01681042C00F098
:1051F0006F81082C00F06C8114F5803F00F068810D
:105200005A6822F4E0625A601123036380F83E502A
:10521000202380F83D30FFF70DFF18E1446C44F087
:105220000104E4B2C1E70469B4F5804F05D190F8F8
:105230003D40212C446CF2D1B5E7046D34B9446C87
:10524000E41104F0060444F0F004AEE7046D012C10
:10525000ACD1446CE41104F0060444F0F104A4E77A
:105260006A4C0C401CB1960501D5446CD9E7684CDA
:105270000C40002C9AD0940598D590F83E40C66A10
:10528000D0F830E090F83D70E4B2222F40F0AF80CB
:10529000076D47B9402C06D100975C6900949C6962
:1052A0000094009C82E7046D8CB90769B7F5404F04
:1052B0000DD101945C6901949C690194019C1C6866
:1052C00044F480741C60046D013404656EE7448D01
:1052D000A4B254B902945C6902949C690294029C41
:1052E0001C6844F400741C6019E0448DA4B2012CC5
:1052F00042D116F5803F1BD11C6824F480641C60E9
:105300005C6814F400640CD01C6824F480641C6095
:10531000002403945C6903949C690394039C002417
:10532000D3E704945C6904949C690494049CD7E7D3
:10533000042E15D0082E13D0BEF1120F10D0C46A5F
:10534000022C1C6814BF24F4806444F480641C6044
:10535000002405945C6905949C690594059CDEE72E
:105360001C6824F480641C60002406945C69069424
:105370009C690694069CB3E7448DA4B2022C23D109
:10538000C46A0026022C1C6814D044F400641C601B
:1053900007965C6907949C690794079C1C6824F431
:1053A00080641C605C682705B9D55C6844F480544F
:1053B0005C60B4E744F480641C6008965C690894FF
:1053C0009C690894089CEDE71C6844F480641C60A8
:1053D0005C68260542BF5C6844F480545C6000242D
:1053E00009945C6909949C690994099C97E70024D5
:1053F0000A945C690A949C690A940A9CD6E600BFE8
:1054000004001000040001008000010008000100F9
:1054100002000100212A03D0402918D1222A16D1E6
:10542000428D92B222B95A6822F480625A600EE02C
:1054300090F83E20402A28D1026D82B9C26C012A20
:10544000826C06D1D2B21A61036D023303650DB0CE
:10545000F0BDC2F307221A61036D0133F6E7026D56
:10546000012A02D1826CD2B2F5E7026D022AEED196
:1054700090F83D20222A04D11A6842F480721A6002
:10548000E5E790F83D20212AE1D1426A511C4162B2
:1054900012781A6199E0002CD9D09405D7D5C16A49
:1054A00090F83D20212AD2D1428D92B2002AECD12F
:1054B00004290DD008290BD011F5803F08D0596878
:1054C00021F4E06159601123036380F83E209FE6D8
:1054D0005A6822F4E0625A601A6842F400721A6054
:1054E00000232022036380F83D2090F83E2080F8BE
:1054F0003E30402A7FF48FAEFFF7A2FDA7E78F4D25
:105500000D40002D46D0510544D5002C42D190F8D5
:105510003D20222A9BD1428D92B2032A05D9426AAC
:105520001B69511C416213704FE0023A012AC26AA2
:105530000DD8022A1A681DBF22F480621A601A6808
:1055400042F4806218BF42F400621A606BE7022ADC
:105550001A6814BF22F4806242F480621A605A68AA
:1055600022F4E0625A60426A1B69511C4162137066
:10557000438D013B9BB24385202380F83D300023BF
:10558000036390F83E2080F83E30402A51D1FFF767
:1055900058FD5CE7002C3FF45AAF97057FF557AFF5
:1055A000C26A418D89B20329416A13D1042A04D009
:1055B000082A02D012F5803F03D11A6822F48062D3
:1055C0001A601B694A1C42620B70438D013B9BB2FF
:1055D00043853CE7448DA4B2022CF2D1042A1FD0AB
:1055E000082A1DD012F5803F1AD0022A1A6814BF6B
:1055F00022F4806242F480621A605A6822F4407297
:105600005A601B694A1C42620B70438D013B9BB27E
:105610004385436A5A1C4262026812691A70A7E7FE
:105620005A6822F440725A601A6842F400721A6092
:10563000E7E7FFF700FD0AE7414C0C4074B196051F
:105640000CD599699B6981F004011D06C1F38001A5
:1056500054BF8289028BFFF7F1FCF8E6394C0C400D
:10566000002C73D0940571D590F83D205968D2B2C2
:1056700021F4E061596000210B9159690B9119687F
:1056800041F0010119600B99196821F480611960DA
:10569000596809050CD590F83D10222903D090F8DF
:1056A0003D102A2929D1816B0968496889B2418551
:1056B000418D89B2E1B159694F0708D5416A1B692B
:1056C0004C1C44620B70438D013B9BB243850168C7
:1056D0004B695E0608D5436A09695C1C446219700F
:1056E000438D013B9BB24385036C43F00403036489
:1056F000036C23B1FFF7A8FCA9E6416BD4E7A2F144
:10570000280102290AD8104AC2622022036380F8C5
:105710003D2080F83E30FFF792FC98E6036B222B89
:1057200002D0222A7FF493AE00232022036380F864
:105730003D2080F83E30FFF780FC88E64000010005
:1057400002000100100001000000FFFF394E3A4C3A
:105750002E400C40002E36D0384D0D403DB355053F
:1057600025D524BB90F83D10428DC9B292B2002AD3
:105770003FF46DAE426A541C446212781A61428D45
:10578000013A92B24285428D92B2002A7FF45FAE16
:1057900029297FF45CAE5A6822F480625A60212382
:1057A0000363282380F83D30FFF746FC4FE6002CCA
:1057B0003FF44DAE94057FF54AAE428D92B2002A79
:1057C0007FF463AE43E61E4D0D4035B3510524D53D
:1057D0001CBB90F83D20418DD2B289B200293FF424
:1057E00036AE416A1B694C1C44620B70438D013B11
:1057F0009BB24385438D9BB2002B7FF428AE2A2AAF
:105800007FF425AE0268536823F48063536022233B
:105810000363282380F83D308DE7002C3FF417AE5A
:1058200092057FF514AE428D92B2002A7FF477AED6
:105830000DE600BF0400100004000100800001001C
:1058400040000100406A08B50368416B1A6822F401
:1058500080621A60002242854A63816B4A6390F835
:105860003D1060294FF0200180F83D1080F83E2067
:1058700007D102641A6822F001021A60FFF7E3FB05
:1058800008BD1A6822F001021A60FFF7DBFB08BDB1
:1058900003682DE9F341DB07054610D42B689F0709
:1058A0005ED42B68190700F195802B685A0700F128
:1058B000BF80EA69002A40F02D81002014E0904C5E
:1058C000636803F00C03042B07D0636803F00C0338
:1058D000082B0CD16368DE0309D523689C03DDD552
:1058E0006B68002BDAD1012002B0BDE8F0816B6853
:1058F000B3F5803F10D1236843F480332360FEF773
:10590000C3FC064623689803C8D4FEF7BDFC801B81
:105910006428F7D90320E7E79BB9236823F4803391
:105920002360236823F480232360FEF7ADFC064642
:1059300023689903B2D5FEF7A7FC801B6428F7D92A
:10594000E8E7B3F5A02F236803D143F48023236055
:10595000D1E723F480332360236823F48023CDE749
:10596000674C636813F00C0F07D0636803F00C03F7
:10597000082B10D16368DA030DD423689B0702D586
:105980002B69012BAFD123686A6923F0F80343EA3E
:10599000C203236085E72A695A4B6AB101221A6063
:1059A000FEF772FC064623689F07ECD4FEF76CFCFA
:1059B000801B0228F7D9ADE71A60FEF765FC0646A2
:1059C000236898077FF56DAFFEF75EFC801B022809
:1059D000F6D99FE7AA694A4C4B4BDAB101221A600B
:1059E000FEF752FC0646636A9B070DD54FF4FA5248
:1059F000464B1B68B3FBF2F3019300BF019B5A1E99
:105A00000192002BF9D150E7FEF73EFC801B0228E3
:105A1000E9D97FE71A60FEF737FC0646636A9F07FD
:105A20007FF543AFFEF730FC801B0228F6D971E703
:105A3000334CE369D80024D40127E36943F0805351
:105A4000E361E36903F080530093009B304E3368B9
:105A5000D90518D5EB68012B26D1236A43F0010341
:105A60002362FEF711FC41F288368046236A9B07C9
:105A70003FD5002F3FF41DAFE36923F08053E3616E
:105A800017E70027E2E7336843F480733360FEF7DB
:105A9000FBFB80463368DA05DCD4FEF7F5FBA0EBB0
:105AA00008006428F6D935E7ABB9236A41F2883893
:105AB00023F001032362236A23F004032362FEF729
:105AC000E3FB0646236A9807D3D5FEF7DDFB801B70
:105AD0004045F7D91EE7052B236A03D143F00403A1
:105AE0002362BAE723F001032362236A23F004034D
:105AF000B6E7FEF7C9FBA0EB0800B042B6D909E74C
:105B0000001002400000424280044242080000208F
:105B100000700040224C636803F00C03082B3FF434
:105B2000E2AE00231F4E022A33602BD1FEF7ACFBFE
:105B30000746236899011FD42B6AB3F5803F05D12E
:105B4000E26AA96822F00F020A43E262696A6268A7
:105B50000B4322F474121343636001233360FEF796
:105B600093FB054623689A013FF5A7AEFEF78CFB31
:105B7000401B0228F6D9CDE6FEF786FBC01B0228A3
:105B8000D7D9C7E6FEF780FB054623689B017FF562
:105B900094AEFEF779FB401B0228F6D9BAE600BFA7
:105BA000001002406000424230B589B06C461B4B89
:105BB00003F11005224618685968083303C2AB4246
:105BC0001446F7D1164B04AC03F1100522461868B1
:105BD0005968083303C2AB421446F7D111494B68E8
:105BE00003F00C02082A17D1C3F3834208A8024429
:105BF000DB0312F8202C0CD5CB6A0B4803F00F0303
:105C0000504308AA134413F8103CB0FBF3F009B05A
:105C100030BD06485043FAE70348F8E7A48300087C
:105C2000B48300080010024000127A0000093D0011
:105C30000268F8B512F0020F05463C4C11D0570728
:105C400042BF636843F4E0636360160742BF636862
:105C500043F4605363606368816823F0F0030B438F
:105C60006360D0071AD42A68510756D4130706D5A3
:105C700063682A6923F4605343EAC2036360FFF751
:105C800093FF63682A4AC3F30313D35CD840294BBC
:105C900018600020FEF7BCFA0020F8BD6868236891
:105CA000012802D19A0305D4F8BD02281BD113F0B4
:105CB000007F39D0636841F2883723F0030318432B
:105CC0006060FEF7E1FA6B680646012B0ED163684F
:105CD00003F00C03042BC6D0FEF7D6FA801BB842A3
:105CE000F5D90320F8BD13F0020FE2E7022B0FD124
:105CF000636803F00C03082BB5D0FEF7C5FA801BD0
:105D0000B842F5D9EDE7FEF7BFFA801BB842E8D8F4
:105D1000636813F00C0FF6D1A5E76368E96823F414
:105D2000E0630B436360A1E70120F8BD001002406F
:105D30000785000808000020044B054A5B68C3F390
:105D40000223D35C034A1068D84070470010024019
:105D50001785000808000020044B054A5B68C3F360
:105D6000C223D35C034A1068D84070470010024039
:105D7000178500080800002003682DE9F341DF07BC
:105D8000064620D5304CE369DD0029D40127E369BC
:105D900043F08053E361E36903F080530193019B77
:105DA0002A4D2B68D8051DD5236A13F440732DD1D5
:105DB000236A726823F44073134323621FB1E369BB
:105DC00023F08053E361306810F002001BD01E4ABC
:105DD000B1685368002023F440430B43536012E042
:105DE0000027DDE72B6843F480732B60FEF74CFA45
:105DF00080462B68D905D7D4FEF746FAA0EB0800F9
:105E00006428F6D9032002B0BDE8F081726802F47C
:105E100040729342CCD001200D4A236A10600020CA
:105E200023F440711060DA072162C1D5FEF72CFA25
:105E300041F288380546236A9B07B9D4FEF724FA55
:105E4000401B4045F7D9DDE70010024000700040DC
:105E50004004424203680020DA6842F00102DA603E
:105E60001A6842F001021A60704770477047704725
:105E70007047036810B51A69044691070ED5DA68B1
:105E800092070BD56FF002021A6101229B6902771B
:105E90009B0777D0FFF7EAFF0023237723681A696F
:105EA000500710D5DA6851070DD56FF004021A615A
:105EB00002229B69227713F4407F204668D0FFF7C7
:105EC000D5FF0023237723681A6912070FD5DA68F4
:105ED00010070CD56FF008021A610422DB692277E3
:105EE000990720465AD0FFF7C1FF00232377236884
:105EF0001A69D20610D5DA68D0060DD56FF01002F7
:105F00001A610822DB69227713F4407F20464BD0C8
:105F1000FFF7ACFF0023237723681A69D10708D560
:105F2000DA68D20705D56FF0010220461A6100F049
:105F300005FE23681A69100608D5DA68110605D52A
:105F40006FF0800220461A6100F0C5F823681A69D4
:105F5000520608D5DA68500605D56FF04002204693
:105F60001A61FFF785FF23681A69910622D5DA685E
:105F700092061FD56FF020022046BDE810401A613E
:105F800000F0A8B8FFF771FF2046FFF770FF83E726
:105F9000FFF76BFF2046FFF76AFF92E7FFF765FF09
:105FA0002046FFF764FFA0E7FFF75FFF2046FFF7FB
:105FB0005EFFAFE710BD0000264A036890420AD09A
:105FC000B0F1804F07D0A2F59432904203D002F591
:105FD0008062904211D14A6823F0700313431D4A36
:105FE000904215D0B0F1804F12D0A2F59432904279
:105FF0000ED002F5806290420AD0174A904207D034
:1060000002F58062904203D002F58062904203D193
:10601000CA6823F4407313434A6923F0800313438F
:1060200003608B68C3620B6883620A4B98420BD093
:1060300003F5A053984207D003F58063984203D03C
:1060400003F58063984201D10B6903630123436127
:10605000704700BF002C01400040014010B50446CD
:10606000A0B190F83D3003F0FF021BB980F83C204E
:1060700001F01EF80223206884F83D30211DFFF74F
:106080009BFF0123002084F83D3010BD012010BD8E
:1060900090F83C3010B5012B4FF0020318D080F877
:1060A0003D3003680C685A68496822F070025A60F3
:1060B0005A6822435A609A6822F080029A609A686D
:1060C0000A439A60012380F83D30002380F83C3079
:1060D000184610BD704770470368DA6822F4907262
:1060E000DA605A6922F001025A61202380F83A30BE
:1060F000704700002DE9F04781460568C2682B69AA
:10610000C16923F4405313432B6183680069EA6833
:106110000343D9F8140022F41642034322F00C0280
:106120000B431343EB606B69D9F8182023F44073D9
:106130001343B1F5004F6B617E4B7FD19D424FF011
:10614000190447D1FFF708FE04FB00F3D9F80470E7
:106150004FF064087F00B3FBF7F3B3FBF8F31F01C4
:10616000FFF7FAFD6043D9F804305B00B0FBF3F6AB
:10617000FFF7F2FD6043D9F804305B00B0FBF3F3A6
:10618000B3FBF8F308FB1363DB003233B3FBF8F324
:106190005B0003F4F876FFF7DFFD6043D9F80420D5
:1061A0005200B0FBF2FAFFF7D7FD6043D9F8043094
:1061B0005B00B0FBF3F3B3FBF8F308FB13A3DB00C6
:1061C0003233B3FBF8F303F007033B443344AB60D3
:1061D000BDE8F087FFF7B0FD04FB00F3D9F80470C9
:1061E0004FF064087F00B3FBF7F3B3FBF8F31F0134
:1061F000FFF7A2FD6043D9F804305B00B0FBF3F673
:10620000FFF79AFD6043D9F804305B00B0FBF3F36D
:10621000B3FBF8F308FB1363DB003233B3FBF8F393
:106220005B0003F4F876FFF787FD6043D9F804209C
:106230005200B0FBF2FAFFF77FFDB6E79D424FF048
:10624000190443D1FFF788FD04FB00F3D9F804607B
:106250004FF06408B600B3FBF6F3B3FBF8F31E018E
:10626000FFF77AFD6043D9F804309B00B0FBF3F7E9
:10627000FFF772FD6043D9F804309B00B0FBF3F3E5
:10628000B3FBF8F308FB13731B013233B3FBF8F3D2
:1062900003F0F007FFF760FD6043D9F80420920097
:1062A000B0FBF2FAFFF758FD6043D9F804309B00C9
:1062B000B0FBF3F3B3FBF8F308FB13A31B0132337A
:1062C000B3FBF8F303F00F033B437FE7FFF734FD25
:1062D00004FB00F3D9F804604FF06408B600B3FB88
:1062E000F6F3B3FBF8F31E01FFF726FD6043D9F880
:1062F00004309B00B0FBF3F7FFF71EFD6043D9F8B5
:1063000004309B00B0FBF3F3B3FBF8F308FB13730B
:106310001B013233B3FBF8F303F0F007FFF70CFD7A
:106320006043D9F804209200B0FBF2FAFFF704FDB5
:10633000BAE700BF00380140F8B504460E461746DC
:106340001D4621680B6836EA030301D10020F8BD21
:106350006B1CF7D095B923680320DA6822F4D07259
:10636000DA605A6922F001025A61202384F8393038
:1063700084F83A30002384F83830F8BDFDF784FF04
:10638000C01B8542DDD2E6E710B5044640B390F865
:10639000393003F0FF021BB980F8382000F09CFE72
:1063A0002423226884F83930D368204623F400532C
:1063B000D360FFF79FFE236800201A6922F4904201
:1063C0001A615A6922F02A025A61DA6842F40052CC
:1063D000DA602023E06384F8393084F83A3010BD65
:1063E000012010BD2DE9F0411F4690F839300446D8
:1063F000202B0D4690464ED1002949D0002A47D087
:1064000090F83830012B46D0012380F83830002333
:10641000C363212380F83930FDF736FF0646A4F820
:106420002480A4F82680E38C9BB26BB93B463246AD
:1064300040212046FFF780FFA8B9202384F83800C8
:1064400084F83930BDE8F081E38C3246013B9BB2E1
:10645000E384A3688021B3F5805F20463B460ED1DC
:10646000FFF76AFF10B10320BDE8F0812B88226896
:10647000C3F308035360236943B90235D3E7FFF739
:106480005BFF0028EFD123682A785A600135CAE7FC
:106490000120BDE8F0810220BDE8F08190F83A309B
:1064A000202B20D1E9B1E2B190F83830012B1AD07D
:1064B000C285828500232222C36380F83A200268C5
:1064C0008162D16880F8383041F48071D1605169BF
:1064D000184641F001015161D16841F02001D160BD
:1064E00070470120704702207047704790F83A309B
:1064F00010B5222B36D183680169B3F5805F02683D
:10650000836A23D15268E9B9C2F3080223F8022B47
:106510008362C48D013CA4B2C4858CB90368DA6877
:1065200022F02002DA60DA6822F48072DA605A69B6
:1065300022F001025A61202380F83A3000F0A4FAD8
:10654000002010BDD2B223F8012BE1E721B9591C7C
:10655000526881621A70DCE75268591C816202F04D
:106560007F02F7E7022010BD70470000036870B596
:106570001A6804461607D9685D6907D196065AD588
:106580008D0658D5BDE87040FFF7B0BF15F0010586
:1065900002D111F4907F4ED0D30705D5CE0542BF6E
:1065A000E36B43F00103E363500704D51DB1E36BD4
:1065B00043F00203E363930704D51DB1E36B43F09B
:1065C0000403E363160704D51DB1E36B43F008032E
:1065D000E363E36B002B66D0950604D5880602D5ED
:1065E0002046FFF783FF236820465D69E26B1107B1
:1065F00002D415F040051AD0FFF76EFD23685A69E2
:10660000520610D55A69606B22F040025A6150B1AF
:10661000254B4363FDF7DEFF002844D0606BBDE8E7
:106620007040436B18472046FFF79EFF70BDFFF791
:106630009BFFE56370BD160627D50D0625D594F89A
:106640003920212A2FD1A268B2F5805F226A17D1A2
:106650001188C1F308015960216979B902322262B7
:10666000E28C013A92B2E284EAB9DA6822F080025E
:10667000DA60DA6842F04002DA6070BD0132EEE7BB
:10668000511C216212785A60EAE750060BD54A067F
:1066900009D5DA68204622F04002DA60202384F827
:1066A0003930FFF722FF70BDAD66000808B5002342
:1066B000406AC385C384FFF757FF08BDF8B5457826
:1066C0000446032D4ED0082D6BD0012D48D13F4FED
:1066D0000679397811B38E423FD12A464FF4807142
:1066E0003B48FEF79FF83B4800F0F4FD00253A4F89
:1066F0003A4E795D3046013500F0ECFD0F2DF8D1B2
:10670000374800F05BFE2946334800F035FA002296
:106710004FF480712E48FEF785F821E0EEB931463E
:10672000304800F0D7FD4FF480712A462848FEF724
:1067300079F8BE232370032304216370E378A170EA
:1067400023713B78E370601C00F0F0FBEB23A17831
:1067500060710331A371C9B21FE0234800F0BAFD94
:106760002046F8BD194D297811B103798B4216D115
:1067700001224FF480711648FEF754F80423637029
:106780002379A178E370601C2B7000F0CFFB29788F
:106790006071164800F09EFD07212046B5E71448B9
:1067A000DCE70A4D02792B789A42D9D14FF48071F7
:1067B00001220748FEF736F8BE232370092304217F
:1067C0006370E378A17023712B78BBE78C00002005
:1067D00000080140C483000896000020D783000809
:1067E0009F840008DD830008F98300080E840008F8
:1067F000288400087FB50023ADF814308DF81630DA
:106800000A230293012305AA8DE80C000A460146DB
:106810000348FEF7EFFA9DF8140007B05DF804FB9B
:10682000500100200A2310B586B006AC04F8012DF3
:10683000029301230A460193014600940248FEF7A1
:1068400043FA06B010BD00BF500100202DE9F74308
:106850000368504DCDF8013043689DF80060CDF8D5
:1068600005309DF806309DF807109DF801E09DF871
:1068700002009DF803709DF804209DF8054041EA50
:1068800003212B784EEA062E47EA002744EA022429
:10689000032B0ED8DFE803F0021023363E4BA3F89B
:1068A00000E03E4B1F803E4B1C803E4B1980012375
:1068B0002B7003B0BDE8F083374B1E88B644A3F8B5
:1068C00000E0364B188807441F80354B1A88144463
:1068D000344A1C801388194411800223E8E72E4BA8
:1068E0001E88B644A3F800E02C4B188807441F808C
:1068F0002B4B1A8814442B4A1C801388194411808E
:106900000323D5E7244BDFF8A4901E8899F8009064
:106910007644B6101FFA86F8A3F800801F4B4FEAA2
:1069200018281888384480101FFA80FCA3F800C08B
:106930001B4B4FEA1C2C1A8822449210194C1FFA48
:1069400082FEA3F800E023884FEA1E2E0B44BE21EE
:106950009B109FB22780144C3F0A2170052166715D
:10696000617000260C21E071601CE372A17084F854
:10697000039084F8048084F806C084F808E062720A
:10698000A772267300F0D2FAEB236073A3732E7004
:106990008FE700BF9200002090000020FA00002046
:1069A000940000208E000020960000208C00002023
:1069B00007B592215220FFF71DFF94215220FFF7C7
:1069C00019FF95218DF801005220FFF713FF962142
:1069D0008DF800005220FFF70DFF97218DF803007E
:1069E0005220FFF707FF98218DF802005220FFF791
:1069F00001FF99218DF805005220FFF7FBFE9A2137
:106A00008DF804005220FFF7F5FE9B218DF807005A
:106A10005220FFF7EFFE8DF806000DF10100FFF7A1
:106A200015FF03B05DF804FB08B5012200215220D8
:106A3000FFF7F8FE0320FDF72DFC03220021522072
:106A4000FFF7F0FE0F4B1B78D52B13D003D8ABB15B
:106A5000C02B11D008BDF62B0AD0FF2B03D0EB2B97
:106A60000FD1322000E00320BDE80840FDF712BC42
:106A70001820F9E76520F7E79A20F5E74FF42F7023
:106A8000F2E708BD480100200268224B10B59A4287
:106A900004461BD1204B21481A782149007888549C
:106AA0001A78D2B2501C8A5CC0B2EB2A187008D196
:106AB0001A788978033A91420ABF01220022194BC1
:106AC0001A70012215491848FFF7E8FC2268174B95
:106AD0009A421DD1164B17481A78114900788854EC
:106AE0001A78D2B2501C8A5CC0B2EB2A187008D156
:106AF0001A788978033A91420ABF02220022094B90
:106B00001A700122BDE810400A490B48FFF7C6BCC5
:106B100010BD00BF00380140360100204A020020AD
:106B2000040100204C010020D80100200044004056
:106B300037010020A40100204C0200200268064B0F
:106B40009A4207D1054A136801331360044A136857
:106B500001331360704700BF0014004000010020A3
:106B6000FC00002010B514460A230248FFF73AFC47
:106B7000204610BDD80100200A460A2301460148DC
:106B8000FFF730BC4C020020F8B5054600231F4C2F
:106B90001F4F2A785E1CDBB29A4220D81D4800F0B5
:106BA0000DFCA1781C4863185A7800F0DAF910BB84
:106BB000174F2B78461CC0B2834216D8A378002109
:106BC0001C446278154800F085FB0021144B2970A5
:106BD00019703222BDE8F8400C4800F073BBE15C4C
:106BE000384600F077FB3346D3E7215C384600F0A7
:106BF00071FB3046DDE7012803D10448FFF75EFD55
:106C0000E3E7084800F0DAFBDFE700BF04010020FB
:106C1000D78300089F8400080501002043840008F2
:106C20004C0100206984000830B593B0282200216F
:106C300008A800F047FB1422002103A800F042FB43
:106C40000123002402250C93102308A80D9300941F
:106C5000019402940895FEF71BFE0F23214603A81A
:106C600003930494059406940794FEF7E1FF6846A5
:106C700000950294FFF780F813B030BD2DE9F04382
:106C800089B0FDF7E9FAFFF7CFFF102200210DEBE5
:106C9000020000F017FB874B4FF400419A698648C9
:106CA00042F010029A619A69002402F010020192E7
:106CB000019A9A694FF0010942F004029A619A69B7
:106CC000022502F004020292029A9A694FF4E13816
:106CD00042F008029A619B69002203F008030393C3
:106CE000039BFDF79FFD00224FF401417348FDF720
:106CF00099FD002238217248FDF794FD4FF40043BE
:106D000004A96D4804930795CDF814900694FDF7F7
:106D1000A9FC4FF4014304A9684804930795CDF8F2
:106D200014900694FDF79EFC38230C27654E04A9A9
:106D3000634804930795CDF814900694FDF792FCF0
:106D4000614B624D304686E808017761B460F460BB
:106D50003461B461F461FFF717FB5D4B284685E8A9
:106D600008016F61AC60EC602C61AC61EC61FFF715
:106D70000BFB40F21F33DFF8B081564A404688E8EB
:106D80000C0009230494C8F80C300594C8F8084096
:106D9000C8F81840FFF762F904A940460494059426
:106DA000FFF776F94C484D494D4B4E4F80E80A00AD
:106DB0004FF4804384600361C46044618461C461B2
:106DC0000462FDF701FF484B38463B604FF46023F7
:106DD000BC60FB61FC607C617C60C7F8109004942F
:106DE00005940694FDF70EFB04A938460494CDF8EB
:106DF00014900694FDF760FA224621462520FDF7FF
:106E000093FB2520FDF7C4FB224621462620FDF7F3
:106E10008BFB2620FDF7BCFB224621463720FDF7E1
:106E200083FB3720FDF7B4FB4046FFF713F84A46D3
:106E30002E493046FFF732FB4A462D492846FFF7D8
:106E40002DFB2C4B21461B682B4F986800F0BEFA97
:106E50002A4800F0B3FA2A4800F0B0FA294A2A4931
:106E60002A4800F037FA2A4800F0A8FA234800F030
:106E7000A5FA284B2848197800F02CFAFFF7D4FD22
:106E8000264D0D4E3C784CB1012C03D12448FFF720
:106E90007BFEF7E7022CF5D12248F8E72B68642B3C
:106EA000F0D9FFF785FD4FF400413046FDF7BFFCF8
:106EB0002C60E7E70010024000100140000801408C
:106EC000000C0140D8010020003801404C02002095
:106ED00000440040001400405001002000540040D5
:106EE000A0860100A8010020002401404A020020E1
:106EF000A40100200C0000204C0100207784000831
:106F0000A1840008B5840008BE840008CA84000873
:106F1000DB8400088C000020F9840008FC000020BD
:106F200036010020370100208C02002010B5FF231D
:106F30000446221AD2B2914201D8184610BD14F864
:106F4000012B5340082213F0800F02F1FF324FEA69
:106F5000430318BF83F0310312F0FF02DBB2F2D11A
:106F6000E7E730B5FF2305462C1AE4B2A14203D867
:106F70009B1A5842584130BD15F8014B6340082414
:106F800013F0800F04F1FF344FEA430318BF83F07E
:106F9000310314F0FF04DBB2F2D1E5E70E4B82B00F
:106FA0009A6942F001029A619A6902F00102009224
:106FB000009ADA6942F08052DA61DB69074A03F02D
:106FC00080530193019B536823F0E06343F0806397
:106FD000536002B0704700BF001002400000014043
:106FE00010B5044686B01022002102A800F06AF90C
:106FF0002268104B9A421BD103F56C439A6902A98F
:1070000042F400729A619A690B4802F4007200928D
:10701000009A9A6942F004029A619B6903F00403A2
:107020000193019B0123029303230393FDF71AFBB2
:1070300006B010BD002401400008014010B5044610
:1070400086B01022002102A800F03CF92268154BFE
:107050009A4224D1144C02A9A369144843F00803AE
:10706000A361A36903F008030093009BC02302936C
:107070001223039303230593FDF7F4FA0022E36937
:107080001F2043F40013E361E369114603F4001386
:107090000193019BFDF748FA1F20FDF779FA06B02E
:1070A00010BD00BF0054004000100240000C014021
:1070B0000268084B82B09A420AD103F5FE33DA69BE
:1070C00042F02002DA61DB6903F020030193019BA7
:1070D00002B0704700140040102210B5044688B07A
:1070E0000DEB0200002100F0EDF82368274A9342DF
:1070F00029D1274B04A99A69264842F480429A6113
:107100009A6902F480420092009A9A6942F004025D
:107110009A619B6903F004030193019B4FF4007390
:1071200004930223059303230793FDF79BFA4FF47F
:1071300080630493002304A9164805930693FDF782
:1071400091FA08B010BD144A9342FAD1104B04A929
:10715000DA69104842F40032DA61DA6902F4003286
:107160000292029A9A6942F004029A619B6903F0C2
:1071700004030393039B0423049302230593032333
:107180000793FDF76FFA0823D3E700BF00380140EB
:107190000010024000080140004400407047FEE734
:1071A000FEE7FEE7FEE7704770477047FDF760B8FF
:1071B0000148FDF7DDBF00BF500100200148FFF787
:1071C000D5B900BFD80100200148FFF7CFB900BFF3
:1071D0004C0200200148FEF74CBE00BF8C0200208C
:1071E0000F4B1A6842F001021A6059680D4A0A40B2
:1071F0005A601A6822F0847222F480321A601A6887
:1072000022F480221A605A6822F4FE025A604FF477
:107210001F029A600022DA62034A044B9A607047A8
:10722000001002400000FFF80040000800ED00E000
:10723000002103E00B4B5B58435004310A480B4BD1
:1072400042189A42F6D30A4A02E0002342F8043B6D
:10725000084B9A42F9D3FFF7C3FF00F00FF8FFF78E
:107260000DFD7047C0850008000000207000002060
:1072700070000020D0020020FEE7000070B500255D
:107280000C4E0D4CA41BA410A54209D101F07EF8B0
:1072900000250A4E0A4CA41BA410A54205D170BDBE
:1072A00056F8253098470135EEE756F825309847CF
:1072B0000135F2E7B8850008B8850008B8850008F0
:1072C000BC85000803460244934200D1704703F88E
:1072D000011BF9E70FB40A4B13B51C6824B1A3696D
:1072E00013B9204600F0DAFA05AB049AA1682046EB
:1072F000019300F09BFC02B0BDE8104004B0704761
:107300000C00002070B50E46054618B183690BB914
:1073100000F0C4FAAB69AC6813B9284600F0BEFAB5
:10732000234B9C4217D16C68A3891B071DD5236989
:10733000DBB1013EA36816F8011F013BA360E9B968
:10734000002B2EDA22460A21284600F0F5F80130FB
:1073500011D00A2070BD174B9C4201D1AC68E3E705
:10736000154B9C4208BFEC68DEE72146284600F03A
:1073700035F90028DDD04FF0FF3070BD002B04DA66
:10738000A269934206DB0A2904D023685A1C2260B2
:107390001970CFE72246284600F0CEF80130C9D157
:1073A000E9E70A2023685A1C2260187070BD00BFEC
:1073B000448500086485000824850008024B0146C6
:1073C0001868FFF79FBF00BF0C00002000294FF492
:1073D00080630CBF0222002200F000B82DE9F743C1
:1073E0001D46514B04461E680F46904626B1B369B0
:1073F00013B9304600F052FA4C4B9C4252D174689B
:10740000B8F1020F06D0B8F1010F00F28980002D0B
:10741000C0F286802146304600F0D6F9616B41B15A
:1074200004F14403994202D0304600F02DFB0023C2
:1074300063630023A3616360A3891B0603D52169ED
:10744000304600F021FBA389B8F1020F23F44A6310
:1074500023F00303A3815DD001AB6A462146304689
:1074600000F0A6FAA3891843A0812DBB009D2846F1
:1074700000F002FB074600284ED1DDF80090A94538
:107480003CD14FF0FF30A38943F00203A3810023D6
:10749000A36004F14703236023610123636103B008
:1074A000BDE8F083224B9C4201D1B468A8E7214B90
:1074B0009C4208BFF468A3E7002FD8D0B36913B982
:1074C000304600F0EBF9B8F1010F08BFA38927603F
:1074D00004BF43F00103A381A389276113F00800CF
:1074E00065611BD013F001004FF000031FBF6D4218
:1074F000A360A561184608BFA560D0E7484600F024
:10750000BBFA07460028BCD0A3894D4643F0800350
:10751000A381D3E70020B6E7A946F5E7A060BEE760
:107520004FF0FF30BBE700BF0C000020448500088F
:107530006485000824850008F8B50E461446054603
:1075400018B183690BB900F0A9F9214B9C422AD1EB
:107550006C68A369A360A3891A072ED5236963B356
:1075600023692068F6B2C01A63693746984204DB83
:107570002146284600F028F928BBA3680130013BCA
:10758000A36023685A1C22601E706369984204D06D
:10759000A389DB0719D50A2E17D12146284600F00A
:1075A00013F990B10FE00B4B9C4201D1AC68D0E7CE
:1075B000094B9C4208BFEC68CBE72146284600F007
:1075C0000DF80028CCD04FF0FF373846F8BD00BF8B
:1075D000448500086485000824850008324B70B596
:1075E0001D6806460C4625B1AB6913B9284600F064
:1075F00055F92E4B9C420FD16C68B4F90C309AB2FD
:1076000015072CD4D00611D40922326043F0400370
:10761000A3814FF0FF3070BD254B9C4201D1AC6877
:10762000EBE7244B9C4208BFEC68E6E7510712D514
:10763000616B41B104F14403994202D0304600F03D
:1076400023FA00236363A38923F02403A381002387
:10765000636023692360A38943F00803A38123693E
:107660004BB9A38903F42073B3F5007F03D02146FF
:10767000304600F0C1F9A28912F001030CD00023BA
:10768000A36063695B42A361236953B9B4F90C3009
:1076900013F08000BAD170BD920758BF6369A36030
:1076A000F2E70020F7E700BF0C0000204485000847
:1076B00064850008248500088A892DE9F041054683
:1076C00010070C465AD44B68002B05DC0B6C002BC2
:1076D00002DC0020BDE8F081E66A002EF9D000232C
:1076E00012F480522F682B6033D0606DA3895A0743
:1076F00005D56368C01A636B0BB1236CC01A0023F5
:107700000246E66A216A2846B047431CA38906D18F
:1077100029681D294BD82B4ACA40D60747D50022D5
:1077200062602269D904226004D5421C01D12B6811
:1077300003B96065616B2F600029CAD004F144036E
:10774000994202D0284600F09FF900206063BDE80E
:10775000F081216A01232846B047411CC6D12B681D
:10776000002BC3D01D2B01D0162B01D12F60B0E709
:10777000A38943F04003A381BDE8F0810F69002F86
:10778000A7D0930718BF00230E6808BF4B69A6EB6C
:1077900007080F608B60B8F1000F9ADD43463A4648
:1077A000216A2846A66AB047002807DCA38943F06F
:1077B0004003A3814FF0FF30BDE8F0810744A8EB00
:1077C0000008E8E70100402038B50B6905460C4683
:1077D000DBB118B183690BB900F060F80C4B9C4227
:1077E00009D16C68B4F90C307BB121462846BDE85C
:1077F0003840FFF761BF074B9C4201D1AC68F1E70D
:10780000054B9C4208BFEC68ECE7002038BD00BF88
:10781000448500086485000824850008014900F0BB
:10782000A9B800BFC9770008002310B5044603605B
:107830004360836081814366C281036143618361E8
:10784000194608225C30FFF73DFD054B2462636258
:10785000044BA362044BE362044B236310BD00BFDF
:10786000A9810008CB810008038200082782000854
:1078700070B568254A1E55430E4605F1740100F0A7
:107880004FF9044640B1002180E842000C30A0606E
:1078900005F16802FFF716FD204670BD836910B53B
:1078A000044633BB8364C3640365124B124A1B68EE
:1078B0008262984204BF0123836100F01FF8606078
:1078C000204600F01BF8A060204600F017F80022C8
:1078D000E06004216068FFF7A7FF01220921A0688A
:1078E000FFF7A2FF02221221E068FFF79DFF0123AC
:1078F000A36110BD208500081D780008F8B51C4B59
:1079000007461E68B36913B93046FFF7C7FF48360C
:10791000B4687368013B03D5336833B13668F7E761
:10792000B4F90C506DB16834F4E704213846FFF720
:107930009FFF30600028F1D10C2304463B602046B5
:10794000F8BD4FF6FF73E38101236566A3812560CF
:10795000A560656025616561A5610822294604F17D
:107960005C00FFF7AFFC6563A563A564E564E6E72B
:10797000208500082DE9F84380468946002600F15D
:10798000480414B93046BDE8F883A5686768013F2C
:1079900001D52468F5E7AB89012B07D9B5F90E307D
:1079A000013303D029464046C84706436835EEE711
:1079B00070B50E46B1F90E1090B0002914461D4660
:1079C00007DA00232B60B3891A0610D44FF48063C2
:1079D0000EE001AA00F04EFC0028F2DB029A02F44D
:1079E0007042A2F500535A425A412A60EEE7402302
:1079F0000020236010B070BD8B8973B59D070646CB
:107A00000C4607D504F1470323602361012363611A
:107A100002B070BD01AB6A46FFF7CAFF0099054688
:107A2000304600F07DF848B9B4F90C309A05EFD42F
:107A300023F0030343F00203A381E3E70D4BB3629A
:107A4000A389206043F08003A381009B20616361D0
:107A5000019B5BB1B4F90E10304600F01DFC28B15B
:107A6000A38923F0030343F00103A381A3891D43EA
:107A7000A581CDE71D780008024B0146186800F08B
:107A80004FB800BF0C00002038B50546002943D090
:107A900051F8043C0C1F002BB8BFE41800F02CFC7C
:107AA0001E4A1368104633B9636014602846BDE867
:107AB000384000F022BCA3420BD9216862189342DF
:107AC00001BF1A685B685218226063600460EDE7CA
:107AD00013465A680AB1A242FAD919685818A04246
:107AE0000BD120680144581882421960DED1106819
:107AF0005268014419605A60D8E702D90C232B6000
:107B0000D4E7206821188A4201BF11685268091819
:107B1000216062605C60C9E738BD00BF38010020A9
:107B200070B5CD1C25F0030508350C2D38BF0C258C
:107B3000002D064601DBA94203D90C233360002047
:107B400070BD00F0D9FB234A1468214691B9224C3C
:107B500023681BB9304600F017FB206029463046E9
:107B600000F012FB431C26D10C233046336000F09A
:107B7000C4FBE4E70B685B1B1AD40B2B0FD90B601B
:107B8000CC18CD50304600F0B8FB04F10B00231D9B
:107B900020F00700C31A1BD05A42E25070BD8C423D
:107BA0000BBF63684B681360636018BF0C46E9E75E
:107BB0000C464968CAE7C41C24F00304A04205D05F
:107BC000211A304600F0E0FA0130CDD02560D9E727
:107BD00070BD00BF380100203C010020936810B444
:107BE000013B002B936008DA9469A34202DBCBB21D
:107BF0000A2B02D110BCFFF79FBC1368581C106001
:107C00001970C8B210BC7047F8B506460F46144646
:107C1000D518AC4201D1002007E03A4614F8011B08
:107C20003046FFF7DBFF431CF3D1F8BD2DE9F04FE1
:107C30009DB00C4617460393064618B183690BB9ED
:107C4000FFF72CFE7C4B9C4257D17468A389180720
:107C50005DD52369002B5AD00023099320238DF88A
:107C6000293030234FF0010B8DF82A30B8464546B5
:107C700015F8013B002B55D1B8EB070A0BD0534642
:107C80003A4621463046FFF7BFFF013000F0C4807E
:107C9000099B5344099398F80030002B00F0BC80F6
:107CA00000234FF0FF3204930793059206938DF85B
:107CB00053301A9305222978604800F00FFB05F134
:107CC0000108049B002831D1D90644BF20228DF839
:107CD00053201A0744BF2B228DF853202A782A2AD2
:107CE0002CD000210A20079AA84698F800300135C8
:107CF000303B092B6DD971B326E0514B9C4201D129
:107D0000B468A3E74F4B9C4208BFF4689EE7214646
:107D10003046FFF763FC00289ED04FF0FF301DB0C7
:107D2000BDE8F08F252BA7D0A846A0E7434A4546DB
:107D3000801A0BFA00F018430490BBE7039A111D58
:107D400012680391002A01DB079204E0524243F0DB
:107D500002030792049398F800302E2B10D198F864
:107D6000013008F101012A2B37D1039B08F10208E9
:107D70001A1D1B680392002BB8BF4FF0FF33059309
:107D8000314D032298F80010284600F0A7FA40B1C0
:107D90004023401B03FA00F0049B08F10108034351
:107DA000049398F800100622284808F101078DF87E
:107DB000281000F093FA002834D0254B03BB039B16
:107DC000073323F0070308330393099B4B440993BC
:107DD0004CE700FB0232012186E700230A25184602
:107DE0000593884698F800200131303A092A03D9D2
:107DF000002BC5D00590C3E705FB00200123F0E769
:107E000003AB00932246134B04A93046AFF3008026
:107E1000B0F1FF3F8146D8D1A3895B063FF57DAF26
:107E200009987CE703AB009322460A4B04A930462D
:107E300000F08AF8ECE700BF44850008848500085C
:107E400064850008248500088A8500088E8500085E
:107E500000000000097C00082DE9F04791461F460C
:107E60008A680B6906469342B8BF1346C9F80030CA
:107E700091F843200C46DDF8208012B10133C9F897
:107E800000302368990642BFD9F800300233C9F8A0
:107E90000030256815F0060507D104F1190AE368DA
:107EA000D9F800209B1A9D422ADB94F843302268BF
:107EB000003318BF012392062FD404F14302394640
:107EC0003046C047013022D02368E56803F006033E
:107ED000042B18BF0025D9F800204FF0000908BF77
:107EE000AD1AA368226908BF25EAE5759342C4BFAD
:107EF0009B1AED181A344D451BD10020BDE8F087C0
:107F00000123524639463046C047013003D14FF075
:107F1000FF30BDE8F0870135C1E73020E11881F876
:107F200043005A1C94F845102244023382F843104F
:107F3000C3E70123224639463046C0470130E6D028
:107F400009F10109D7E700002DE9F04317460A7E41
:107F500085B06E2A984606460C460C9B01F1430EEE
:107F600000F0BC801AD8632A2ED00AD8002A00F06C
:107F7000C880582A00F08A8004F1420584F8422023
:107F80002AE0642A01D0692AF6D121681A6811F022
:107F9000800F23D0111D1960136827E0732A00F0A9
:107FA000B48008D86F2A2AD0702AE5D10A6842F036
:107FB00020020A6003E0752A21D0782ADCD17822D9
:107FC0006F4984F8452064E01A6801F14205111DEB
:107FD0001960136884F842300123A3E011F0400FC8
:107FE00002F104011960D7D0B2F90030002B03DA96
:107FF0002D225B4284F8432062490A2217E0206860
:10800000196810F0800F03D0081D18600B6806E097
:1080100010F0400F01F104001860F7D00B886F2AB0
:1080200014BF0A2208225749002084F843006568DB
:10803000002DA560C0F29C80206820F00400206024
:10804000002B3FD1002D40F095807546082A0BD1BA
:108050002368DA0708D5236962689A42DEBF3023B5
:1080600005F8013C05F1FF35AEEB05032361CDF8C2
:1080700000803B4603AA21463046FFF7EDFE013063
:1080800055D14FF0FF3005B0BDE8F08381F84520B1
:108090003C492268186812F0800F00F104051D6049
:1080A00001D0036802E05506FBD50388D00744BF22
:1080B00042F0200222601BB9226822F020022260D6
:1080C0001022B1E77546B3FBF2F002FB1033CB5C34
:1080D00005F8013D03460028F5D1B7E708681A689E
:1080E00010F0800F496904D0101D186013681960E2
:1080F00007E010F0400F02F1040018601368F6D09A
:108100001980002375462361B1E71A68111D1960B3
:10811000156800216268284600F0E0F808B1401BAD
:10812000606063682361002384F843309FE723691C
:108130002A4639463046C0470130A2D023689B0703
:1081400007D5002504F11909E368039A9B1A9D429B
:1081500005DBE068039B9842B8BF184693E701230C
:108160004A4639463046C04701308AD00135EBE7F0
:10817000002BA7D10B7804F1420584F8423065E763
:10818000A68500089585000838B50023054C0546EE
:108190000846236000F0ECF8431C02D1236803B1C9
:1081A0002B6038BDCC02002010B50C46B1F90E1082
:1081B00000F0A4F80028ABBF636DA3891B1823F45B
:1081C0008053ACBF6365A38110BD2DE9F0411F460C
:1081D0008B890546DB050C46164605D50223002291
:1081E000B1F90E1000F068F8A389324623F48053E9
:1081F000A381B4F90E103B462846BDE8F04100F0DB
:1082000017B810B50C46B1F90E1000F055F8431C24
:10821000A38915BF606523F4805343F48053A38181
:1082200018BFA38110BDB1F90E1000F013B8000003
:1082300038B50546084611460022054C22601A460C
:10824000FEF790FC431C02D1236803B12B6038BDBC
:10825000CC02002038B50023054C054608462360B3
:1082600000F05EF8431C02D1236803B12B6038BDD7
:10827000CC02002038B50023064C054608461146BE
:10828000236000F055F8431C02D1236803B12B6032
:1082900038BD00BFCC02002038B50023054C054690
:1082A0000846236000F04CF8431C02D1236803B158
:1082B0002B6038BDCC02002038B505460846114673
:1082C0000022054C22601A4600F042F8431C02D1FD
:1082D000236803B12B6038BDCC02002010B5C9B2B1
:1082E00002449042034601D1002010BD1C780130A9
:1082F0008C42F6D1184610BD7047704738B5054618
:10830000084611460022054C22601A4600F028F863
:10831000431C02D1236803B12B6038BDCC0200207E
:108320005822024B4FF0FF301A607047CC020020F9
:108330005822024B4FF0FF301A607047CC020020E9
:108340005822024B00201A60704700BFCC02002068
:108350005822024B4FF0FF301A607047CC020020C9
:108360005822024B4FF0FF301A607047CC020020B9
:10837000044B0246196809B9034919601868024498
:108380001A60704740010020D0020020F8B500BFFD
:10839000F8BC08BC9E467047F8B500BFF8BC08BCE6
:0483A0009E4670473E
:1083A40002030405060708090A0B0C0D0E0F101032
:1083B4000102030405060708090A0B0C0D0E0F1031
:1083C4004D5920524742205374617475732053658C
:1083D4006E64002530327820004D592049442049EC
:1083E40053204E4F5420534554203A2025303278A0
:1083F40020200D0A004E4F204D5920494420495356
:10840400202530327820200D0A004D79204944205F
:108414005345542053756363657373202530327854
:10842400200D0A004D7920494420616C656164790E
:108434002065786973742025303278200D0A004F46
:10844400726967696E616C20435243203A2025307B
:1084540032782052656376435243203A20253032E5
:1084640078200D0A00576861742048617070656E49
:108474003F0D002A2A2A2A2A2A2A2A2A2A2A2A2A8A
:108484002A2A2A2A2A2A2A2A2A2A2A2A2A2A2A2A48
:108494002A2A2A2A2A2A2A2A2A2A2A0D0052474222
:1084A4002053656E736F722050726F6A6563740D2A
:1084B4000031393A31343A32340041707220313269
:1084C4002032303139004275696C64206174202592
:1084D400732025730D0A00436F707972696768749D
:1084E4002028632920323031392E20424C5545430F
:1084F400454C4C0D004D79204944202530327820DC
:108504000D0A000000000000000000010203040640
:108514000708090000000001020304001000002005
:108524000000000000000000000000000000000047
:108534000000000000000000000000000000000037
:108544000000000000000000000000000000000027
:108554000000000000000000000000000000000017
:108564000000000000000000000000000000000007
:1085740000000000000000000000000000000000F7
:10858400232D302B2000686C4C00656667454647F8
:10859400003031323334353637383941424344457B
:1085A40046003031323334353637383961626364EA
:0485B40065660000F8
:0485B800F541000881
:0485BC00D1410008A1
:1085C000010000001000000000366E0110000020C5
:1085D0000000000044850008648500082485000828
:1085E000000000000000000000000000000000008B
:1085F000000000000000000000000000000000007B
:10860000000000000000000000000000000000006A
:10861000000000000000000000000000000000005A
:10862000000000000000000000000000000000004A
:04000005080072314C
:00000001FF
